:020000040000FA
:080000000528000000000000CB
:08000800D9288C012100093008
:100010008C00240008308C00210000309900200062
:1000200000308C00230001308C0021000F3095003F
:1000300000308B0021000030910021000030920040
:1000400064002100183097006400210001309D00F9
:100050002100F3309E002200823097002000003003
:100060009C00220000309100220000309200250008
:100070000330960020005E28000021001D1420009F
:10008000DA20A201A3014030A4000130A000A00B9F
:10009000472821009D149D184B2821001B08200093
:1000A000A2070318A30A21001C082000A307A40B21
:1000B0004528230821001D1020000800FF30A5005E
:1000C0000430A6008C0102218C1600000C160000E2
:1000D0008C14EE208C1200000C1200008C10E42016
:1000E0000C1502217E20E420EE208C1D7E20A50B25
:1000F0007A28C720A6080319D22874280C16F820DD
:100100000C1200008C1600008C14F8208C120000D9
:100110008C1000000C16F8203C200C12A800F820CF
:100120002808833C031CB3281030A70028087D3C16
:1001300003189B28AB28A70B9E28BC288C16000010
:100140000C1600008C14EE208C1200000C12000023
:100150008C10EE209B28A70BAE28BC288C16EE2016
:100160008C12EE20AB288C162808893C031C0C1638
:100170002808903C031C8C14EE208C1DBC280C21FC
:100180000C218C1200000C1200008C100800FF30B3
:10019000A5003C207D3C0318D0280430A6000800B0
:1001A000A60308000C11E42063000000000000001A
:1001B000742809000130A1001930A000A00BDE282E
:1001C000A10BDE28640008000130A1008330A000EC
:1001D000A00BE828A10BE828640008000230A10069
:1001E0000830A000A00BF228A10BF2286400080040
:1001F0000430A1001C30A000A00BFC28A10BFC289F
:10020000640008000630A1003030A000A00B0629D1
:10021000A10B0629640008000B30A1006230A00089
:0C022000A00B1029A10B1029640008009D
:04022C000034003466
:100280005034493443342034423461347434743447
:10029000203463346F346E34743472346F346C349D
:1002A00043346F3470347934723469346734683469
:1002B00074342834433429343234303431343534CE
:1002C000203456342E3431342034203442346F34C8
:1002D000723467344D3463347A342034203420341B
:1002E00062346F34723467346D344034733465343F
:1002F0007A346E3461346D342E3463347A3420347D
:020000040001F9
:08000000003400340034023426
:02000E00840F5D
:02001000FF1AD5
:00000001FF
